S31508001800E0080020D9180008E7180008E9180008B9
S3150800181000000000000000000000000000000000BA
S315080018200000000000000000000000000119000888
S315080018300000000000000000031900083137000806
S3150800184011400008071900080719000807190008B9
S3150800185007190008071900080719000807190008DA
S315080018600719000899280008071900080719000829
S3150800187007190008071900080719000807190008BA
S3150800188007190008000000000000000007190008FA
S3150800189000000000071900080719000807190008C2
S315080018A0000000000719000807190008753B000822
S315080018B007190008071900080719000800000000A2
S315080018C0EE11AA550348854600F030FC004800474B
S315080018D01D520008E00800200B4880F308880B48D2
S315080018E080470B480047FEE704207146084202D0AD
S315080018F0EFF3098001E0EFF30880714603F012FB6D
S31508001900FEE7FEE7FEE7FEE7E0080020C537000829
S31508001910C518000830B50B460146002020220124D0
S3150800192009E00D46D5409D4205D31D469540491B05
S315080019302546954040191546521E002DF1DC30BD4E
S3150800194070B500242546002801DA01244042002902
S3150800195001DA01254942FFF7DDFFAC4200D04042DB
S31508001960002C00D0494270BD03460B439B0703D0A9
S3150800197009E008C9121F08C0042AFAD203E00B7846
S315080019800370401C491C521EF9D27047D2B201E0BE
S315080019900270401C491EFBD270470022F6E710B5BC
S315080019A013460A4604461946FFF7F0FF204610BDBF
S315080019B0F8B502464A40D40F42004B0052085B086D
S315080019C09A4202D20246084611464A0023D0C30D5F
S315080019D04A00DDB2120EAD1A202D35DA490201266B
S315080019E0490AF6058A19002C00D0524220214F1BBD
S315080019F01146B9402A411018C20D9A4221D0002C2E
S31508001A0017D0012D08DCDA05801AD20F8019D20703
S31508001A10DBB200F0F2FAF8BDDA05801A01234000BD
S31508001A201B06C01880185A428018CA0F104349006E
S31508001A3007E04908C2071143DA05801A80194008E9
S31508001A40801800F0D2FAF8BD61000122511A001B75
S31508001A50F7E70122D2075140AAE70122D2075040F0
S31508001A60A6E7024670B54A40D30FDB0740002DD0E3
S31508001A704A002AD0010E140E000212020919400A61
S31508001A80520A8418E50104465443000A120A2E0431
S31508001A905043A4194219200CC543AA18120C012553
S31508001AA0AD03521C521912047F39240400D0521C6B
S31508001AB0104301D44000491EC2B20C06C0092018C2
S31508001AC0401C4008802A02D003E0002070BD400870
S31508001AD04000002900DA0020184370BD70B50246A0
S31508001AE04A40D50F40004A00ED0740085208002832
S31508001AF014D0002A12D0C40DD30D41020120C0050E
S31508001B005202490A520AE41A091812187D349142F7
S31508001B1001D3641C00E04900002C01DA002070BDE6
S31508001B200023914201D3891A03434008490000283B
S31508001B30F7D100290AD0914202D10121C90705E04F
S31508001B40914201D2012101E00121C943E005C018F3
S31508001B50401900F04AFA70BDF0B5074608465840E5
S31508001B6087B0C00F049048000E465900400849083F
S31508001B70BC1A884105D2384631461E4617460B46DA
S31508001B8002465800400810434CD0300D03904005DB
S31508001B905900400D490D0590401A0290402872DA06
S31508001BA018030121000B09050843019004980092C7
S31508001BB0002805D0019952420020884100920190E0
S31508001BC0029840210A1A0199009800F0EBF9054697
S31508001BD00C466B4607CB00F0F5F9C0197141039A1C
S31508001BE00E0D0023D71756401A467A40164344D09E
S31508001BF0049A002A2DD0029A012A039A15DC1205A6
S31508001C00C01A914101263605001C7141D20F059E66
S31508001C10D2070093019202962A46234600F033FA29
S31508001C2007B0F0BD38463146FAE71605224A0F4690
S31508001C30B218C01AB74101210905001C4F41001806
S31508001C407F41114618187941E20F10436D19644116
S31508001C5013E0E2076D0815436408C2071443039AA4
S31508001C6001261205C01A91413605001C7141CE079E
S31508001C70400830434908C01851412A46234600F017
S31508001C80F5F9CDE7FFE7049801224000C117121ABB
S31508001C9000238B4104983146C417381AA141EEE750
S31508001CA030B40124E407634030BC55E730B401245E
S31508001CB0E407614030BC4FE70000E0FFF0B51FB411
S31508001CC088B00B990998002448400999C00F490023
S31508001CD049080991C0070B990090490049080B91DA
S31508001CE009990898A64608431CD00B990A980843F0
S31508001CF018D0099801244000420D4800410D099862
S31508001D0024050003000B204309900B980003000BE1
S31508001D1020430B9050181C49401800220190144685
S31508001D20104605E0002001460DB0F0BD032801DA93
S31508001D30034600E003239C46C11A0AAE0AE05F0088
S31508001D4008ADED5B4F00F75B7D430027AA187C4181
S31508001D50491C5B1E6145F2DD410004AB5A52210461
S31508001D60120C0A43240C401C0828DFDB0198029059
S31508001D700099704601910090059B049A0799069868
S31508001D8000F081F9D0E700000DFCFFFFF0B50C4626
S31508001D905C4085B0E40FE40703944C000026640811
S31508001DA059009446490802460296224321D06246C3
S31508001DB00A431ED06200570D4A000E032303550D31
S31508001DC0012402462C492405781B1B0B360B4018A8
S31508001DD023432643614600901C46501AB44103D358
S31508001DE00098401C009002E0921800985B41002879
S31508001DF003DA0020014605B0F0BD002001210905DF
S31508001E000746864611E064461D46141BB54106D3AF
S31508001E106546521BB341744607430C43A646CD0795
S31508001E2040084908284392185B4105460D43EAD104
S31508001E301046184313D0604619465040714008436F
S31508001E4006D06046101AB34106D20122002306E0E6
S31508001E5000220123DB0702E00122D2435310009837
S31508001E6074460105381C6141029C039D00196941AD
S31508001E7000F0FCF8BFE70000FD030000C217C10F21
S31508001E80504010B54018CA079623002100F0B5F84F
S31508001E9010BD10B500229623114600F0AEF810BD0D
S31508001EA00EB505490291002100910A460B4601919B
S31508001EB000F0E9F803B000BD330400004100400219
S31508001EC00122400AD205090E80187F2901DA00206E
S31508001ED07047962903DC9622511AC84070479639EE
S31508001EE088407047C20FD207400040080BD0C10D8A
S31508001EF00723DB01C91840020905400A1143C20835
S31508001F00400711437047002001467047CB0FDB0797
S31508001F10490010B5490802460A4307D00A0D0724A6
S31508001F200903E401090B121B002A01DC002010BD7D
S31508001F30C900440F0C43C100E018D205801800F010
S31508001F4054F810BDF0B51FB40646002082B0054609
S31508001F504024019100901BE0019922460F46304625
S31508001F6000F0F6F8049A059B801A994110D310469A
S31508001F701946224600F016F8361A8F41019722466E
S31508001F8001200021009F00F00DF838184D410090FF
S31508001F902046641E0028DFDC019B0098294632464D
S31508001FA007B0F0BD10B5202A04DB0146203A91405F
S31508001FB0002010BD914020239C1A0346E340194394
S31508001FC0904010BD10B5202A06DBCB170846203AEC
S31508001FD01041C1170B4306E00B461341D04020249D
S31508001FE0A21A91400843194610BD002904DA401C7C
S31508001FF0490001D140084000704770B40024050C20
S3150800200005D11024000402D1002921D01124050E7F
S3150800201001D100020834050F01D10001241D850FE6
S3150800202001D18000A41C002801DB4000641C0029A3
S3150800203008D020252E1B0D46F540A14000D00121D1
S315080020402943084301061B1B000ADB1D02D5002095
S3150800205070BC7047DB05181880180029F8DA401C90
S315080020604900F5D170BC40084000704710B5002BF8
S3150800207008DA0024401C614192185B411A4301D1D9
S315080020804008400010BDF0B51FB482B005460C00EC
S3150800209003D0084602F00AF802E002F007F82030FA
S315080020A00246009021462846FFF77CFF049B059AC6
S315080020B004460F4618431143084314D018461043E4
S315080020C01BD0009840210A1A1846059900F040F8D6
S315080020D005460E46009A05990498FFF763FF0843DC
S315080020E005D0012004E02046394607B0F0BD00209F
S315080020F0C11705430E432C43374300990E986305D1
S31508002100401A7905E40A00220C43FD0A0A3002D572
S3150800211000200146E9E70105101969410C9C0D9D4F
S3150800212000196941FFF7A2FFDFE70000064C012509
S31508002130064E05E0E36807CC2B430C3C9847103461
S31508002140B442F7D3FFF7C2FBA85D0008C85D0008D4
S3150800215010B5202A04DB0846203AD040002110BDDD
S315080021600B46D340D0402024A21A91400843194672
S3150800217010BD000010B50446002C08D10121092025
S31508002180C00600F037FE002000F05AF94BE0012C9B
S3150800219005D102210920C00600F02CFE43E0022CDE
S315080021A005D104210920C00600F024FE3BE0032CDB
S315080021B005D108210920C00600F01CFE33E0042CD6
S315080021C005D110210920C00600F014FE2BE0052CCD
S315080021D005D120210920C00600F00CFE23E0062CBC
S315080021E005D140210920C00600F004FE1BE0072C9B
S315080021F005D180210920C00600F0FCFD13E0082C5B
S3150800220004D101210A4800F0F5FD0CE0092C04D19F
S315080022100221074800F0EEFD05E00B2C03D1102142
S31508002220034800F0E7FD204600F00AF910BD00005B
S3150800223000040048FEB5002000900190029000249A
S31508002240A3E000250DE006206843654940186100B3
S31508002250405AA1006A4651584018A1005050681CBF
S3150800226085B2142DEFDBA1006A4650581421FFF7FA
S3150800227051FB2821484361005A4A515A3C2251438E
S31508002280461864213046FFF745FB6100554A50520F
S3150800229055480079002806D160001146085AA10061
S315080022A0524A50506EE0012C01D0022C6AD14E4899
S315080022B02038407E002808D1012C06D16000494903
S315080022C0085AA100494A50505DE0A00047490858FD
S315080022D06100444A515A88422AD260001146085A77
S315080022E0A100424A5158401A0A2817D94048015DA8
S315080022F0005D401C3E4A1055142908DD0020114691
S31508002300085560003749085AA100384A5050A000BD
S315080023103649085A6100334A505233E0002034499E
S31508002320085560002F49085AA100304A505029E044
S31508002330A0002E49085861002A4A515A401A0A280C
S3150800234017D92B48015D005D401C294A10551429F0
S3150800235008DD00201146085560002249085AA100E8
S31508002360224A5050A0002149085A61001D4A50527D
S3150800237008E000201E49085560001A49085AA100BD
S315080023801A4A505000BF601C84B2032C00DA58E782
S3150800239015480079002822D01248408815498842F5
S315080023A003DC10488088884208DD0F482038407DC5
S315080023B0002803D101210C48203841750948408876
S315080023C00A2803DB074880880A2808DA06482038DE
S315080023D0407D002803D10121034820384175FEBD00
S315080023E05403002014010020D4020020CC0300204E
S315080023F021010020E60F000000B587B001A800F013
S31508002400AFF80121480201F005F80020019070207C
S31508002410029001208002039000200690059001A9F1
S31508002420064800F031F80121044800F021F801219E
S31508002430024800F011F807B000BD00000024014072
S3150800244010B50446072300222146024800F038F852
S3150800245010BD000000240140002904D04268012371
S315080024601A43426003E042685208520042607047CD
S31508002470002904D0826808231A43826003E0826830
S3150800248008239A438260704742680B4B1A404260A1
S315080024900B684A681A4343681A4342608268074BC6
S315080024A01A4082600B694A691A438B681A43836823
S315080024B01A438260704700000FBCFFFF8FF1F9FFD7
S315080024C0F0B504460D4616461F463F073F0F2B46F6
S315080024D0082B0FD91B071B0F083B606F9A000F21AB
S315080024E0914088436067606F99003A468A40104376
S315080024F060670BE0206F9A000F21914088432067A0
S31508002500206F99003A468A4010432067E068012107
S31508002510A9408843E060E0680121A9400843E060DB
S31508002520012080032840002803D0012000F020F86D
S3150800253007E00120C0032840002802D0012000F04F
S3150800254017F8F0BD002905D08268FF2301331A4326
S31508002550826004E08268FF2301339A4382607047F1
S31508002560002101604160816001730161416170472A
S31508002570002806D0064949680C221143044A5160CE
S3150800258005E0034949680C229143014A51607047A6
S315080025900024014010B523480078012835D10020D1
S315080025A0204908702049088013E01F480088400029
S315080025B01E49095A1E480088062250431D4A80189B
S315080025C0194A12885200815217480088401C164939
S315080025D00880154800880328E7DB7E2001F024FDE3
S315080025E0022000F02BF901211348FFF7ABFF104832
S315080025F00088401C0E49088008460088142804DB19
S315080026000020088001200D4908700C480078002831
S3150800261006D0FFF70FFE00200849087000F034FCCA
S3150800262010BD0000200100203A01002020030020F0
S315080026303C01002054030020002401401A01002018
S31508002640FFB583B00C46029400200190002726E0CF
S3150800265000261CE0721C039951430846791CFFF7B3
S3150800266059F90546A54201D9281B00E0601B054615
S315080026700298A84204D9029505980670069807702C
S315080026800298002802D10120019002E0761C402E13
S31508002690E0D300BF0198002800D002E07F1C042F79
S315080026A0D6D300BF029807B0F0BD000000BF00BF38
S315080026B000BF00BF00BFBFF34F8F00BF00BF00BF02
S315080026C006480749C86000BF00BF00BFBFF34F8F69
S315080026D000BF00BF00BF00BF00BFFDE70400FA054A
S315080026E000ED00E010B500F001F810BD10B5234864
S315080026F00078002817D1224800F014FF01283CD1A1
S315080027001F480078002838DD1D480078402834DC4A
S3150800271001F003FA1B4908600120184908700020D7
S315080027201949087029E0164A17490978491C5018AA
S3150800273000F0F8FE012816D113480078401C12490B
S3150800274008700F4800780978884216D100200B498E
S3150800275008700B484078FF280FD10B4800780228EC
S315080027600BD1FFF7A3FF01F0D8F9064909686431D0
S31508002770884202D900200149087010BDED000020EA
S31508002780DC020020F0000020EC00002010B586B026
S3150800279004460121880300F03DFE0121480400F0AB
S315080027A019FE01220921C80600F00FFB01220A21A1
S315080027B00920C00600F009FB01A801F0B4FA01944B
S315080027C030216846018100214181818101821821D9
S315080027D0C18101A9184801F063FA0121164801F0E0
S315080027E03CFA05A800F047FB0121490268468182A8
S315080027F0012181751821C17505A90920C00600F0B7
S3150800280097FA01218902684681824821C17505A97E
S315080028100920C00600F08CFA1B21684601700321C6
S3150800282041700121817000F0A1FD012202210248B8
S3150800283001F02BFA06B010BD0038014001B5044975
S315080028400098086000BF024800680028FBD108BD50
S31508002850F4000020014600220E4B1A61CA005A6194
S3150800286000229A6105221A6100BF0A4A1069C20746
S31508002870D20F002A04D0012212040240002AF4D002
S31508002880044A126952085200024B1A6100229A61E0
S315080028907047000000E000E010B500210448FFF78B
S315080028A051FE022000F04AF801200249087010BDC6
S315080028B0002401402001002000B589B00121084606
S315080028C000F088FD1A4800F045F801A800F08EF8D7
S315080028D018480190184802900021684601730320A1
S315080028E0049068460175802141754900C1828900B6
S315080028F0018320218176090281830021C183018415
S3150800290001A90B4800F04CF80121094800F01CF811
S3150800291001220221064800F039F8092168460170AB
S31508002920022141700121817000F020FD09B000BD2F
S3150800293008000240002401402003002001494860A5
S3150800294070470000000002400268520852000A431D
S315080029500260704710B504462068400840002060B1
S31508002960002020606060A060E060E1B20846083898
S315080029700521FEF7CFFF01460F2088400249496826
S3150800298008430149486010BD00000240002A03D0F0
S3150800299003680B43036002E003688B4303607047D8
S315080029A010B50A7A8B7D1A430B7C1A434B7C1A4363
S315080029B04B8A1A438B8A1A430B8B1A434B8B1A433F
S315080029C00368094C23401A43026002680123DB03AB
S315080029D09A438B8B1A430260CA6842600A6882600F
S315080029E04A68C26010BD00000F80FFFF0021016029
S315080029F041600172C16001744174418281828175AE
S31508002A00018341838183704770B506460C4621468B
S31508002A100A4800F02DF90546002D01D1401E70BD6B
S31508002A200648854202D10648051B00E02D1B2246B2
S31508002A3029463046FEF798FF2046F0E700F40008DE
S31508002A4000FC000870B506460C4621460A4800F008
S31508002A500FF90546002D01D1401E70BD0648854276
S31508002A6002D10648051B00E02D1B224629463046A2
S31508002A70FEF77AFF2046F0E7008000080088000885
S31508002A8070B505460C4622460249284600F0B1F8BC
S31508002A90204670BD00F4000870B505460C4622466F
S31508002AA00249284600F0A5F8204670BD00800008B7
S31508002AB010B504460848006902210843064908611A
S31508002AC008464461006940210843034908610348F0
S31508002AD000F00EF910BD000000200240FF0F0000B4
S31508002AE00C48C068C007C00F002801D001207047F5
S31508002AF00848C06804210840002801D00220F6E7EB
S31508002B000448C06810210840002801D00320EEE7D9
S31508002B100420ECE7002002400348006980210843AE
S31508002B2001490861704700000020024030B504469C
S31508002B300D460548006901210843034908612580B7
S31508002B400F2000F0D5F830BD0020024010B57E20D9
S31508002B5001F06AFA064800F00FF87E2001F064FAE0
S31508002B60044800F009F87E2001F05EFA10BD000066
S31508002B7000F400080080000810B5044600F0ACF820
S31508002B802046FFF795FFFFF7C7FF10BD70B5034650
S31508002B900125002208E050001C5A0748844201D04B
S31508002BA0002506E0501C82B2CE0F761876109642A3
S31508002BB0F1DC00BF284670BDFFFF0000F8B50546EA
S31508002BC00E46144600F088F87E2001F02DFA0027FC
S31508002BD007E029883046FFF7A9FFB61CAD1C781C0C
S31508002BE087B2E10F09194910B942F2DCFFF794FFE1
S31508002BF0F8BDF8B507460C4615462946204600F0A6
S31508002C0037F80646002E0DD12046FFF7B5FF0120FE
S31508002C1080022018FFF7B0FF2A4621463846FFF7FC
S31508002C20CDFF24E0012080022018401BB0420AD1C3
S31508002C30012080022018FFF79FFF2A4631463846B2
S31508002C40FFF7BCFF13E00120C0022018401BB0426A
S31508002C5008D12046FFF790FF2A4631463846FFF747
S31508002C60ADFF04E02A4631463846FFF7A7FFF8BD10
S31508002C70F8B505460E462F46E807C00F002801D0CE
S31508002C8000BFFEE731460120C002FEF759FE0029C3
S31508002C9001D000BFFEE700240BE020467043471929
S31508002CA031463846FFF772FF012800D108E0601C5C
S31508002CB084B231460120C002FEF742FEA042ECDC97
S31508002CC000BF31460120C002FEF73AFEA04200D1FD
S31508002CD000273846F8BD0000024803494860034803
S31508002CE0486070472301674500200240AB89EFCD55
S31508002CF010B5024600BFFFF7F3FE0346521EFF2437
S31508002D0000E0641E002CFCD1012B01D1002AF2D16F
S31508002D100648006977218843044908613420C86059
S31508002D20002A01D1052010BD1846FCE70020024004
S31508002D30F8B50246CD782F073F0FCD7810263540D7
S31508002D40002D01D08D782F431446002011E085060A
S31508002D502B0E0D88012686403540002D07D02568A4
S31508002D600F269E40B5433E469E4035432560451C8A
S31508002D70E8B20828EBDB141D0D882D1200950020FB
S31508002D8011E085062B0E01258540009E3540002D55
S31508002D9007D025680F269E40B5433E469E403543DC
S31508002DA02560451CE8B20828EBDBCD78282D04D130
S31508002DB055690E883543556106E0CD78482D03D10F
S31508002DC015690E8835431561F8BD70B54D07EB0ECC
S31508002DD0082902DA0546203501E0054624352C4641
S31508002DE00F269E402568B54316469E403543256006
S31508002DF070BD000038B504460D460920C006844259
S31508002E0003D10121480400F0E5FA1148844203D1B0
S31508002E100121000200F0DEFA0E48844203D10121A6
S31508002E20000200F0D7FA0C48844203D101210805B4
S31508002E3000F0D0FA684600F01EF8684605800121C1
S31508002E4081700021C17069462046FFF771FF38BDC1
S31508002E500004004800080048000C00480246906834
S31508002E600840002801D0012070470020FCE7416196
S31508002E707047016170470021C943018002218170B2
S31508002E800421C17070470000F0B58FB000250026F8
S31508002E9000200D900C907E2001F0C6F800241AE060
S31508002EA06100B44A505AFEF7F4FFB3490790FEF79B
S31508002EB015FE0746FFF716F80022B04B0991089051
S31508002EC0FEF7FCFE0B910A90FFF720F8A100AC4A2A
S31508002ED05050601C84B2032CE2DBA9498868FFF7CE
S31508002EE001F8A84AA84B05910490FEF7D9FE0022DE
S31508002EF0A64B07910690FEF749FFA54AA54B0991EF
S31508002F000890FEF7D3FE0B910A90FEF7FFFF0546E1
S31508002F109B494868FEF7E6FF9F4AA04B0591049037
S31508002F20FEF7BEFE0022994B07910690FEF72EFF8C
S31508002F30974A984B09910890FEF7B8FE0B910A90AC
S31508002F40FEF7E4FF06462846FEF7CCFF00228B4B29
S31508002F5005910490FEF7AAFE099108902946904823
S31508002F60FEF77FFD0746FEF7BDFF07910690099B12
S31508002F70089AFEF70BFF0B910A90FEF7C7FF8949DF
S31508002F8008603046FEF7AEFF00227C4B05910490A0
S31508002F90FEF78CFE0991089031468148FEF761FDDF
S31508002FA00746FEF79FFF07910690099B089AFEF7CA
S31508002FB0EDFE0B910A90FEF7A9FF7B4908607B4955
S31508002FC0088BFEF76DFF7A4A7A4B03910290FEF75B
S31508002FD075FE0022784B05910490FEF7D7FE0991FD
S31508002FE008907249088BFEF754FF0746FEF77AFFEA
S31508002FF00022714B01910090FEF7C8FE05910490DE
S3150800300068480068FEF76EFF03910290059B049AD4
S31508003010FEF746FE07910690099B089AFEF7B6FE4C
S315080030200B910A90FEF772FF0D906049488BFEF7E8
S3150800303037FF5F4A5F4B03910290FEF73FFE00227F
S315080030405D4B05910490FEF7A1FE0991089057493A
S31508003050488BFEF71EFF0746FEF744FF0022564B35
S3150800306001910090FEF792FE059104904E48006883
S31508003070FEF738FF03910290059B049AFEF710FEAF
S3150800308007910690099B089AFEF780FE0B910A9015
S31508003090FEF73CFF0C9049480D99FEF789FC074658
S315080030A0FEF70CFF4649086044480C99FEF780FC79
S315080030B00746FEF703FF434908603C48D830008DB1
S315080030C03F4909684018C003010C3848D8300185C3
S315080030D0408D3C4909684018C003010C3348D83074
S315080030E04185274908683849FEF7BBFC0746FEF7BD
S315080030F0E5FE81B22D48D83081852030C07D002874
S315080031002DD12A48D830808DFD2804DC0021274897
S31508003110F830817312E02548D830808DFF211731A9
S31508003120884205DC01212148F8308173C17505E024
S3150800313002211E48F83081730121C1751B48F830F9
S31508003140017E007E401CC2B21848F83002760F296C
S3150800315001DD0121C175002014492839486013484A
S3150800316028380088642803DD00201049283908809B
S315080031700FB0F0BD1401002000F07F4500000840A4
S31508003180480300209A9999999999C93F00002840BF
S3150800319025068195438BD43F333333333333C33FCB
S315080031A000004843280100202C010020BC01002013
S315080031B0091B9E5E29CB703F00408F400000C84126
S315080031C030010020340100200000C8420148006890
S315080031D070470000F8000020034800680349097892
S315080031E04018014908607047F800002000010020D7
S315080031F008B50121480400F0EDF80121880400F023
S31508003200E9F86846FFF737FE0121C90368460180D9
S315080032104821C17069460920C006FFF789FD68463E
S31508003220FFF729FE01210903684601804821C1707C
S3150800323069460920C006FFF77BFD6846FFF71BFEB7
S315080032404021684601800421C17069460148FFF79C
S315080032506FFD08BD0004004810B50121C903092007
S31508003260C006FFF7FBFD002808D12148807E00280C
S3150800327008D101211E488176C17403E000211C484B
S31508003280C17481761B4880687D21090188422CD942
S3150800329000201849886000211548C174203000793B
S315080032A000281CD108211448FFF7E3FD1048807B4D
S315080032B000280CDD0E482038408D822804DA0121CA
S315080032C00B482030017102E0012109484175084880
S315080032D0807C012809D100200649486005E00020C5
S315080032E0044948600021024881740148C07C10BD29
S315080032F0B4020020940100200004004808B501210A
S31508003300480400F067F80121880400F063F868466D
S31508003310FFF7B1FD0D21684601800121817010215A
S31508003320C17069461048FFF703FD8E216846018083
S31508003330012181701021C17069460920C006FFF776
S31508003340F7FC08210920C006FFF791FD8021092016
S31508003350C006FFF78CFD01210348FFF788FD082109
S315080033600148FFF786FD08BD00040048817800295A
S3150800337025D0174903221202891802789210920062
S31508003380895802789207D30EFF229A4091434278D1
S315080033909207120E03789B07DB0E9A4011430C4ADC
S315080033A003231B02D21803789B109B00D150017887
S315080033B0CA06D20E01219140054A116007E001783C
S315080033C0CA06D20E01219140014A80321160704727
S315080033D000E100E0002905D0054A52690243044B82
S315080033E05A6104E0024A52698243014B5A617047A6
S315080033F000100240002905D0054AD2690243044B51
S31508003400DA6104E0024AD2698243014BDA61704705
S3150800341000100240002905D0054A92690243044B70
S315080034209A6104E0024A92698243014B9A617047A5
S315080034300010024010B500F031F804494968F0223E
S3150800344011400909024A515CC84010BD00100240EB
S31508003450C800002010B5FFF7EDFF054949680722A7
S3150800346012021140090A034A515CC84010BD000007
S3150800347000100240C800002010B5FFF7DBFF054921
S3150800348049680722D2021140C90A034A515CC8405A
S3150800349010BD000000100240C8000020F8B51E4804
S315080034A040680C210840042802D008282ED101E0E3
S315080034B01A4C2DE0184840300069C007C00F002894
S315080034C00AD015484030006902210840002801D07A
S315080034D0134802E0114800E0104807460E484030FD
S315080034E00069FF2109040840000C451C0A484030C1
S315080034F00069072109020840000A461C3946694343
S3150800350008463146FEF706FA044601E0034C00BFBA
S3150800351000BF2046F8BD00000010024000127A00E5
S3150800352000093D0070B5044600250221074800F051
S315080035309AFB002808D0054800F0EEFB207002210F
S31508003540024800F088FB0125284670BD0038014076
S3150800355010B500F001F810BD00B585B062480068E6
S31508003560012108436049086000BF5F4800680221DE
S3150800357008400028F9D05D485D4908605D48006844
S31508003580102108435B49086008460068C008C00067
S31508003590086057490968481E5749FEF7BBF9049061
S315080035A05448006804994907490F08435149086077
S315080035B04D484068514908404B49486008464068AC
S315080035C0902108434849486008464068486048488A
S315080035D000684649884207D94348406805210902D8
S315080035E00843414948600BE041480068444988421D
S315080035F006D93D4840680121890208433A4948608E
S315080036006B4601AA3A4801683E48FFF719F836485A
S315080036104030006980088000334940310861084617
S315080036200069400840000861684600784007400F76
S315080036300290684600794006400E03902A48C06901
S31508003640890508432849C8612748403000692E493A
S315080036500840254940310861039800040299090287
S31508003660084321494031096908431F494031086127
S315080036701D4800680121090608431B49086000E047
S3150800368000BF194800680121490608400028F7D0FC
S315080036901548406880088000134948600846406815
S315080036A0022108431049486000E000BF0E48406800
S315080036B00C2108400828F8D10120FFF7CBF80A4862
S315080036C0406810218843084948600120FFF7C2F87E
S315080036D00548406880218843034948600120FFF770
S315080036E0B9F805B000BD00000010024000A24A0467
S315080036F0D80000200020024000366E010FC0FFFFF0
S315080037000051250200127A00FFF800FF042806D1AE
S315080037100649096904221143044A116105E003496F
S31508003720096904229143014A1161704700E000E0EB
S3150800373010B5FFF751FD20480088401C1E49088037
S3150800374008464068401C48601C480068002804D0A9
S315080037501A480068401E194908601948C07C0128A3
S315080037600CD1174820300079002801D11249486049
S3150800377011488068401C1049886002E000200E4904
S3150800378088600F48007C012805D10B480069401C59
S315080037900949086102E00020074908610848807D58
S315080037A0012805D10448006A401C0349086202E062
S315080037B000200149086210BD94010020F400002091
S315080037C0B402002010B516480068012108431449C0
S315080037D00860084640681349084011494860084689
S315080037E00068114908400E4908600846006801212A
S315080037F0890488430A49086008464068C3210904C1
S31508003800884307494860084600680849084004494B
S3150800381008609F2000048860FFF79AFE10BD00002C
S31508003820001002400CC0FFF8FFFFF6FEFFFF8F00F6
S3150800383008B501214804FFF7CDFD02220121092020
S31508003840C006FFF7C2FA0221684601801821C17036
S315080038500121817069460920C006FFF769FA01212E
S315080038604804FFF7B7FD022211460920C006FFF7F4
S31508003870ACFA0421684601801821C17001218170C3
S3150800388069460920C006FFF753FA08BD30B587B068
S3150800389004460D4601210846FFF7ACFD04A800F0D2
S315080038A033F905946846058200210183817681747F
S315080038B004A90120800700F0F1F8684600F0D2F864
S315080038C060216846017001214170002001900021A5
S315080038D06846017269460120800700F057F8694674
S315080038E00120800700F08AF80821C80600F07EF853
S315080038F00821C80600F0B0F84021080600F038F89C
S315080039004021080600F03CF80121880700F00AF873
S315080039100121880700F01EF80121880700F00EF83B
S3150800392007B030BD002904D0026880231A4302601C
S3150800393003E0026880239A4302607047002904D096
S31508003940026801231A43026003E002685208520023
S3150800395002607047002905D0426C0123DB031A4335
S31508003960426404E0426C0123DB039A4342647047D5
S31508003970826907231B039A430B021A438261704725
S31508003980C26970239A430A43C261704710B58269B7
S3150800399007231B039A430B781B021A4382610A7A90
S315080039A012014B781B011A43036A3024A3431A43B6
S315080039B002624A6882630C4A904213D14A7A12011B
S315080039C08B781B011A43036AC024A3431A43026275
S315080039D04A8992008B899B001A4343682401A343B2
S315080039E01A43426010BD0000002C01408269012381
S315080039F0DB029A430B021A438261704710B5C2690B
S31508003A0070239A430B781A43C2610A7A12024B78DA
S31508003A101B021A43036A03242402A3431A430262BD
S31508003A204A68C2630B4A904213D14A7A12028B78CB
S31508003A301B021A43036AA400A3431A4302624A8973
S31508003A4012018B891B011A434368A400A3431A4336
S31508003A50426010BD002C0140C26908239A430A43FC
S31508003A60C261704700210170417081704160017226
S31508003A70417241818181704701229207904201D1AA
S31508003A80816301E08AB282637047012292079042FD
S31508003A9001D1C16301E08AB2C26370470268032399
S31508003AA01B029A430B891A430260134A904206D0B6
S31508003AB001229207904202D0104A904205D102682C
S31508003AC070239A438B781A4302600B4A904205D0BA
S31508003AD00B4A904202D00B4A904205D1026B120A59
S31508003AE012028B7A1A4302634A68C2620A888262A1
S31508003AF00122426170470000002C0140000400408A
S31508003B0000440140004801400021C94341600021AA
S31508003B100180018181708172704710B5FFF756FBED
S31508003B2010BD000070B5FFF785FC05467D21C9006C
S31508003B30FDF7F0FE0446601E0C49884200D90CE0E9
S31508003B40601E0B4948610321081F00F0D5FA0020C2
S31508003B50074988610720086100BF0420FFF7D6FDE2
S31508003B600021481E00F0C8FA70BD0000FFFFFF00E4
S31508003B7000E000E010B50221154800F07DF80028A5
S31508003B8024D0134800F0C8F8C4B21248007C0028B4
S31508003B9003D1204601F07EF814E00E48007C022886
S31508003BA010D10C48407C00280CD10B488079AA28F3
S31508003BB004D10948C471012106484174AA2C01D1CF
S31508003BC0054884710221024800F045F810BD00003E
S31508003BD000380140B4020020D803002010B504467E
S31508003BE02146054800F09CF800BF0121024800F074
S31508003BF03AF80028F9D010BD0038014070B50546DE
S31508003C000E4600247E2000F00FFA00BF20E0042CA8
S31508003C1019DD701EA04216DD285D7E2806D17D209E
S31508003C20FFF7DCFF5E20FFF7D9FF0FE0285D7D2850
S31508003C3005D1FFF7D3FF5D20FFF7D0FF06E0285D2B
S31508003C40FFF7CCFF02E0285DFFF7C8FF601C84B2CF
S31508003C50B442DCDB70BD416170478269520852008C
S31508003C600A4382617047024690680840002801D0DE
S31508003C70012070470020FCE70246D068084000286B
S31508003C8001D0012070470020FCE7002A03D0036911
S31508003C900B43036102E003698B430361704700002D
S31508003CA070B504460D460026E06930218843297917
S31508003CB00843E061E06944218843A9790843E06143
S31508003CC0E06980088000297A0843E061A069182124
S31508003CD0884369890843A061A06904218843297B30
S31508003CE00843A0610B48844203D1FFF7C5FB06468B
S31508003CF002E0FFF7AFFB064630462968FDF70AFEE5
S31508003D000009206230462968FDF704FE0007000F07
S31508003D10606270BD0038014001464868C0B270470D
S31508003D20CAB2026070474B21C90101603021017196
S31508003D3000218171017218214181002101737047A8
S31508003D4010B5A248807B030000F0C7F905045A8D18
S31508003D50D4F5F4009D482038808DFD280DDB9B485E
S31508003D60F838808B012805D100219848F8388183D6
S31508003D7000F05AFF01219548817340219448FFF7C6
S31508003D806DF8002815D093494868FF21F531FDF7ED
S31508003D90C1FDC007C00F002805D180210920C00633
S31508003DA0FFF765F822E080210920C006FFF761F8D1
S31508003DB01CE088494868C821FDF7ACFDC007C00F5C
S31508003DC0002805D180210920C006FFF750F80DE02C
S31508003DD080494868C821FDF79DFDC007C00F002827
S31508003DE004D080210920C006FFF743F808210920DE
S31508003DF0C006FFF73CF801217548FFF738F8E2E0FE
S31508003E0072482038808DFF211731884202DB022153
S31508003E106E48817340216E48FFF720F8002813D0BA
S31508003E206C494868FF21F531FDF774FDC007C00FDE
S31508003E30002804D101216648FFF719F808E0012196
S31508003E406348FFF716F803E001216148FFF711F808
S31508003E5080210920C006FFF70AF808210920C006B4
S31508003E60FFF705F8AFE059482038808DFF21253146
S31508003E70884202DD03215548817340215448FEF7E4
S31508003E80EDFF002827D053494868FF21F531FDF793
S31508003E9041FDC007C00F00280ED180210920C006A9
S31508003EA0FEF7E7FF01214A48FEF7E3FF082109204C
S31508003EB0C006FEF7DEFF1CE080210920C006FEF7DB
S31508003EC0D6FF08210920C006FEF7D1FF0121404888
S31508003ED0FEF7CDFF0DE080210920C006FEF7C9FFD9
S31508003EE001213B48FEF7C5FF08210920C006FEF759
S31508003EF0C0FF68E040213648FEF7B0FF002843D0EF
S31508003F00012109030920C006FEF7A8FF002813D1DE
S31508003F1080210920C006FEF7ACFF01212C48FEF7D8
S31508003F20A8FF08210920C006FEF7A3FF0421274899
S31508003F30817337E046E036E026494868FF21F531C7
S31508003F40FDF7E8FCC007C00F00280ED18021092024
S31508003F50C006FEF78EFF01211D48FEF78AFF0821DD
S31508003F600920C006FEF785FF1CE080210920C0064F
S31508003F70FEF77DFF08210920C006FEF778FF01211C
S31508003F801348FEF774FF0DE080210920C006FEF7EE
S31508003F9070FF01210E48FEF76CFF08210920C006B4
S31508003FA0FEF767FF0FE080210920C006FEF761FFD4
S31508003FB001210748FEF75DFF08210920C006FEF724
S31508003FC058FF00E000BF00BF10BD0000B40200208B
S31508003FD00004004894010020034880684008400017
S31508003FE00149886070470000002C00408021014389
S31508003FF0014A116070470000002C004003488068A1
S31508004000002801D0012070470020FCE7002C004062
S3150800401010B5FFF7F3FF002804D0FFF7DDFF662091
S3150800402000F002F810BD00004106490E014A116071
S3150800403070470000002C004004494968FF2281327D
S3150800404091430143014A516070470000002C00402B
S3150800405004494968C909C9014206520E1143014A71
S3150800406051607047002C004070B505460C4601218A
S31508004070C802FFF7BFF9FF208130FFF7DDFF2046B2
S31508004080FFF7E6FF2846FFF7B1FF70BD0FB410B57E
S3150800409003A9044B044A029800F07AF810BC08BC3D
S315080040A004B01847714C0008900100202021020C2A
S315080040B001D010211046020A01D01046083902091B
S315080040C001D01046091F820801D01046891E4208F1
S315080040D001D0881E7047081A704730B47446641EAB
S315080040E02578641CAB4204D3635D5B00E31830BCDF
S315080040F018471D46F8E7000010B5002819DB1A4ACC
S3150800410003231B02D21883089B00D2588307DC0EB0
S31508004110FF23A3409A438B071B0E8407E40EA34094
S315080041201A43114B032424021B198408A4001A51AC
S3150800413018E00E4A03071B0F083B9B089B00D25842
S315080041408307DC0EFF23A3409A438B071B0E8407C5
S31508004150E40EA3401A43054B0407240F083CA408A1
S31508004160A4001A5110BD000000E100E01CED00E0BB
S3150800417002E008C8121F08C1002AFAD17047704722
S31508004180002001E001C1121F002AFBD17047000080
S31508004190FFB58FB00F460446002606E025280AD04C
S315080041A0129A11999047641C761C20780028F5D13C
S315080041B0304613B0F0BD00250121A14A009500E064
S315080041C00543641C23780846203B98401042F7D1E3
S315080041D020782E2815D1042005436078641C2A28E7
S315080041E00AD101CF641C00900BE000990A225143C2
S315080041F030394018641C0090207801463039092966
S31508004200F3D920786C280ED004DC4C2813D06A2801
S3150800421012D104E074280ED07A280DD10BE00120C3
S315080042204005054307E00121090562780D438242EE
S3150800423001D16D18641C641C2078864669284AD00A
S3150800424008DC0028B4D058286DD0632810D064281C
S3150800425008D140E070286BD0732812D0752860D03A
S31508004260782860D0129A704611999047761CE5E036
S315080042703878694608720020487202A80190012021
S3150800428003E0386801900020C0433F1D69070CD53C
S31508004290002500E06D1C00998D420FDA8542F9DB96
S315080042A00199495D0029F5D108E0002500E06D1C5B
S315080042B08542FCDB0199495D0029F8D1761907E0AA
S315080042C0019801990078491C0191129A1199904711
S315080042D06D1EF5D2B2E00A20029000216802400F56
S315080042E0039102280CD001CFC117844600290DDAA4
S315080042F06246084652420021814194462D2008E034
S31508004300FF1DFF08FF0003CF8446EFE7280504D505
S315080043102B206A46107401203CE0E8073AD020209A
S31508004320F7E70A2000E0102000210391029007E039
S3150800433010200290002104200543082003910090D4
S315080043406802400F022810D001CF002184460020C1
S315080043500D9028071FD5704670280CD0029A102099
S31508004360039B42401A430CD015E0FF1DFF08FF00CF
S3150800437003CF8446EBE740206A46107401200D906F
S315080043800CE06046084306D030206A461074704632
S31508004390507402200D907046582804D029A0019028
S315080043A00DA80E900DE02CA0F9E76046039B029A33
S315080043B0FDF7C8FD019B84469B5C0E9A521E0E9221
S315080043C0137060460843F0D10E9805A9081A2030E4
S315080043D00190680701D5009801E001200090019935
S315080043E0884203DD01460198081A00E000200025EE
S315080043F0009006E004A8129A405D119990476D1C3A
S31508004400761C0D988542F5DB04E0129A3020119946
S315080044109047761C0099481E00900029F5DC08E0B4
S315080044200E980E990078491C0E91129A1199904788
S31508004430761C0199481E01900029F1DC641CB4E63B
S31508004440092801003031323334353637383961625C
S315080044506364656600000000303132333435363720
S3150800446038394142434445460000000010B502462B
S315080044700023002901D1002010BD03E01488921CF6
S31508004480E01883B208464C1EA1B20028F6D1184699
S31508004490F2E70000F8B50027002600240025F848B2
S315080044A0407C01286FD17E20FFF7BEFDF548C07914
S315080044B00002F449097A08430746F248467A847A9C
S315080044C00246D17A107B00F021FD05460021EC4812
S315080044D04174ED49781A8F426FD01EDCEB49781A81
S315080044E08F426BD010DCEA49781A8F4267D006DC17
S315080044F0442F1CD0E7483818002872D1DCE18828F8
S3150800450070D08928F9D16CE101286CD002286BD0CB
S3150800451003286AD00428F0D135E10300FFF7DDFD52
S315080045200C61C0FAF861611926768E415C61062E27
S3150800453009D1D948007800280AD100F0D7FF012010
S31508004540D549087004E0152E02D1012000F0CEFFEF
S31508004550D0E1CB4820300079002806D0C84820385A
S31508004560028D418D002000F01BFFC3E1002C0BD10A
S31508004570C3482038408D00231A46F0210090FE20BB
S3150800458000F043FF0CE0B6E1012C09D1BC48203805
S31508004590008D01230022F0210090FE2000F035FF57
S315080045A0A8E1002C0CD1BD48408D00231A46F32102
S315080045B00090FE2000F029FF0DE05AE053E189E162
S315080045C0012C08D1B548808E01230022F3210090E2
S315080045D0FE2000F01AFF8DE1002C07D1AF48458573
S315080045E006E086E111E11AE16AE07AE0AB488586E1
S315080045F0AA48808EFF21F531884206DA00F014FBBE
S315080046000022FE21F42000F034FF73E1002C09D1CA
S31508004610A248808D00231A46F1210090FE2000F062
S31508004620F4FE0AE0012C08D19C48C08E0123002222
S31508004630F1210090FE2000F0E8FE5BE1002C02D19B
S315080046409648858503E0012C01D19448C586934890
S31508004650808DFF21F53188420ADC9048C08E884259
S3150800466006DC00F0E1FA0022FE21F22000F001FF4C
S3150800467040E1002C09D18948C08D00231A46E9215A
S315080046800090FE2000F0C1FE09E0012C07D1192098
S3150800469001230022E9210090FE2000F0B6FE29E160
S315080046A0002C01D17D48C585FF202D30854206DACC
S315080046B000F0BAFA0022FE21EA2000F0DAFE19E13B
S315080046C0002C0CD17548008E6421484380B2002323
S315080046D01A46E2210090FE2000F097FE00E000BF97
S315080046E008E1002C06D164212846FDF729F981B294
S315080046F06A4801866948008EFF21F531884206DC42
S3150800470000F092FA0022FE21E32000F0B2FEF1E06A
S315080047101EE0FFE7002C0CD16048408E6421484318
S3150800472080B200231A46EB210090FE2000F06DFEB1
S315080047300DE0012C0BD15948008F6421484380B203
S3150800474001230022EB210090FE2000F05EFED1E05E
S31508004750002C07D164212846FDF7F2F881B24F48AC
S31508004760418608E0012C06D164212846FDF7E8F8C1
S3150800477081B24A48018700F057FA0022FE21EC2050
S3150800478000F077FEB6E0012C13D13D48807B002867
S3150800479006DD01213A482030017100203F49486072
S315080047A00022FE21E42000F064FE012134488174D1
S315080047B016E0002C0FD10021314881742030017198
S315080047C00022FE21E42000F054FE00203249087041
S315080047D03249486004E00022FE21E42000F049FE48
S315080047E088E0002C0FD12748C07A32280CDC2548EF
S315080047F0C17A2A48418700F017FA0022FE21DF20F5
S3150800480000F037FE00E000BF74E02448408F002324
S315080048101A46DE210090FE2000F0F7FD6AE0002C23
S315080048200FD11848C07A32281CDC1648C17A1B48B2
S31508004830818700F0F9F90022FE21E12000F019FE37
S3150800484010E0012C0ED10F48C07A32280ADC0D4838
S31508004850C17A1248C18700F0E7F90022FE21E1205B
S3150800486000F007FE46E0002C1AD10C48808F002382
S315080048701A46E0210090FE2000F0C7FD1BE000006C
S31508004880B4020020D8030020E9FE0000E0FE000084
S3150800489056FE0000AB01FFFF8C01002094010020AA
S315080048A0012C08D11448C08F01230022E021009072
S315080048B0FE2000F0AAFD1DE0002C07D101210F48BB
S315080048C00174002202210E48FFF7DFF90DA0FFF759
S315080048D0DDFB0FE0002C0BD1FF2101310A48FDF763
S315080048E05CF800200849891F0880022103480174E2
S315080048F000E000BF00BFF8BD94010020B40200200C
S315080049000038014031323300DE030020F0B589B0AB
S3150800491000200890079006903D48407C012874D1F5
S315080049203C488079AA286DD13A48C079322869DA94
S315080049303848C079002865DD3649C97908461938E6
S31508004940FDF79CFA08900898FDF7CCFA0446324A17
S31508004950324BFDF7B3F90022314B01910090FDF778
S31508004960FBF8039102902F480068FDF7BBFA06464C
S31508004970039B029AFDF70AFA05910490FDF7C6FA19
S31508004980079029490798FDF76CF80446FDF796FA4B
S3150800499081B21F48F83801830898FDF7A3FA06463E
S315080049A01D4A1E4BFDF78AF9044600221C4BFDF7EB
S315080049B0D3F8039102901D480068FDF793FA019118
S315080049C00090039B029AFDF7E1F905910490FDF723
S315080049D09DFA069014490698FDF743F80446FDF734
S315080049E06DFA81B20A48F838418300F01DF9084883
S315080049F0F838428B018B0EA0FFF748FB00210448CC
S31508004A000174817400210248417409B0F0BD0000A8
S31508004A10B4020020D8030020091B9E5E29CB703FF4
S31508004A200000F03F2801002000007A442C010020F5
S31508004A30525F30203A202025642020525F313A20E8
S31508004A4020202564200D0A0070B505460E4614463A
S31508004A50002E02D0012E52D128E0002D02D0012DC1
S31508004A6022D110E027480078A0420BD0602101200F
S31508004A708007FEF77DFF002101208007FEF7FCFF77
S31508004A802048047010E020480078A0420BD060212E
S31508004A9001208007FEF774FF002101208007FEF73A
S31508004AA0F4FF1948047000BF00BF28E0002D02D0AB
S31508004AB0012D22D110E013480078A0420BD06021C6
S31508004AC001208007FEF754FF214601208007FEF7E4
S31508004AD0D3FF0C48047010E00B480078A0420BD0B6
S31508004AE0602101208007FEF74BFF21460120800741
S31508004AF0FEF7CBFF0448047000BF00BF00BF00BF2D
S31508004B0070BD00003E0100203F01002070B505255C
S31508004B102BE080213648FCF740FF80213448FDF71A
S31508004B2073FF0F213248FFF7A1FC3149C98B884230
S31508004B300CD12F482838008D2E49884204D000F021
S31508004B408DFA00F071F800E070BD0EE02AA0FFF7BC
S31508004B509DFA002407E061002548425A214629A00B
S31508004B60FFF794FA641C802CF5DB2846691ECDB243
S31508004B700028CED100BF05252DE080211C48FCF772
S31508004B800CFF80211A48FDF75DFF0F211848FFF733
S31508004B906DFC1749C98B88420ED115482838008DF7
S31508004BA01449884204D000F059FA00F03DF802E0B2
S31508004BB000F03AF8C8E70EE015A0FFF767FA0024F8
S31508004BC007E061000A48425A214614A0FFF75EFA38
S31508004BD0641C802CF5DB2846691ECDB20028CCD192
S31508004BE000BF00F03BFA00F01FF800BFACE700007A
S31508004BF0BC010020FBAA00004641554C54215F31F8
S31508004C00000000002564202025640D0A200000000D
S31508004C104641554C54215F32000000005F3225643E
S31508004C20202025640D0A200010B57E20FFF7FCF928
S31508004C30FDF78CFF0C480D4908850F210B482830D5
S31508004C40FFF714FC09492831C88380210748283012
S31508004C50FDF716FF7E20FFF7E7F980210348283085
S31508004C60FDF71AFF10BD0000FBAA00009401002002
S31508004C7070B504460D46E1B20548FFF751F800BF86
S31508004C8001210348FEF7EFFF0028F9D0204670BD42
S31508004C900038014070B50446002599480088FA286E
S31508004CA00ADD00209649088096490870FF210131DF
S31508004CB09348801DFCF771FE924800780300FFF7C1
S31508004CC00CFA08052031425BD5EFEDEC7E2C11D1AC
S31508004CD000208B49088001208A4908708848018885
S31508004CE00088401C864A1080901D445400201146B6
S31508004CF0C87002E0002082490880002080490871B7
S31508004D00FBE07F4801880088401C7D4A1080901D82
S31508004D10445402207B490870104600790019114650
S31508004D200871EAE0764801880088401C744A1080B9
S31508004D30901D4454032073490870104600790019E1
S31508004D4011460871D9E06E4801880088401C6C4AF3
S31508004D501080901D445404206A4908701046007952
S31508004D600019114608710846C470C078002802D197
S31508004D70052064490870C0E061484079012856D189
S31508004D805E2C1CD15E4800797E305D4908717E2113
S31508004D905B4802880088401C594B1880981D81542E
S31508004DA0801FC078401EC0B21946C870002802DCB1
S31508004DB005205449087000205149487155E05D2C7A
S31508004DC01CD14F4800797D304D4908717D214C48EA
S31508004DD002880088401C4A4B1880981D8154801F01
S31508004DE0C078401EC0B21946C870002802DC0520EB
S31508004DF04449087000204249487136E04048007925
S31508004E0000193F490871084601880088401C3C4A39
S31508004E101080901D4454801FC078401EC0B21146B1
S31508004E20C870002821DC0520364908701DE07D2C55
S31508004E3003D101203249487117E031480079001939
S31508004E402F490871084601880088401C2C4A1080A2
S31508004E50901D4454801FC078401EC0B21146C870C9
S31508004E60002802DC05202749087046E02448007916
S31508004E70C043401CC5B2A54203D10620214908708B
S31508004E8002E007201F4908701D4801880088401C59
S31508004E901B4A1080901D44542FE02DE01DE0FFE7CB
S31508004EA0174801880088401C154A1080901D4454F4
S31508004EB07E2C08D10121144841740020114608802F
S31508004EC01049087008E000200D49088000210E48A6
S31508004ED0417400200B4908700FE00020094908704A
S31508004EE0074801880088401C054A1080901D4454D4
S31508004EF000201146088000E000BF00BF70BD00001A
S31508004F00D80300208B010020B402002070B50246A9
S31508004F10002013460C461D02FF263602354025435F
S31508004F20284670BD86B004460D4626686768A068A0
S31508004F300590E06804902069039060690290A06972
S31508004F400190E069009017A0FFF7A0F831461BA072
S31508004F50FFF79CF839461CA0FFF798F81DA005999D
S31508004F60FFF794F81EA00499FFF790F81FA003997D
S31508004F70FFF78CF820A00299FFF788F823A001997B
S31508004F80FFF784F826A00099FFF780F82948416AB8
S31508004F9029A0FFF77BF829462BA0FFF777F800BF73
S31508004FA0FEE700005B48617264206661756C7420D8
S31508004FB068616E646C65725D0D0A00005230203DB2
S31508004FC02025780D0A0000005231203D2025780D55
S31508004FD00A0000005232203D2025780D0A00000004
S31508004FE05233203D2025780D0A0000005231322028
S31508004FF03D2025780D0A0000537461636B656420B3
S315080050004C52203D2025780D0A0000005374616338
S315080050106B6564205043203D2025780D0A0000006A
S31508005020537461636B656420505352203D20257884
S315080050300D0A000000ED00E05343425F5348435316
S31508005040523D25780D0A000043757272656E74200C
S315080050504C52203D2025780D0A00000000B5154861
S3150800506015490885FF21144841850F210186A0218D
S31508005070C185D22181851E214186AF21C1868C2119
S315080050800187BE2181860D49283001830B492331CA
S3150800509041830521283841870A218187C187002154
S315080050A0283081830F21FFF7E1F903492831C883A6
S315080050B000BD0000FBAA0000940100205A2500004C
S315080050C010B55348C07D002800D110BD5048407D1A
S315080050D0012826D14F494868C821FCF71BFCC007A0
S315080050E0C00F002805D180210920C006FDF7BFFEA4
S315080050F00DE048494868C821FCF70CFCC007C00FFA
S31508005100002804D080210920C006FDF7B2FE082138
S315080051100920C006FDF7ABFE01213F48FDF7A7FEB3
S31508005120D3E73B48807C01286FD139482030007985
S31508005130002802D001282BD102E0FEF701FE63E029
S3150800514034494868FF21F531FCF7E4FBC007C00F76
S3150800515000280ED180210920C006FDF78AFE01210C
S315080051602D48FDF786FE08210920C006FDF781FEB9
S315080051700DE080210920C006FDF779FE08210920E7
S31508005180C006FDF774FE01212348FDF770FE3BE0DB
S315080051901F4820300079052827D11E494868FF2175
S315080051A0F531FCF7B7FBC007C00F00280ED18021E8
S315080051B00920C006FDF75DFE01211748FDF759FED7
S315080051C008210920C006FDF754FE1CE080210920AD
S315080051D0C006FDF74CFE08210920C006FDF747FE6C
S315080051E001210D48FDF743FE0DE080210920C00688
S315080051F0FDF73FFE01210848FDF73BFE082109207F
S31508005200C006FDF736FE00BF00BF00BF5DE7000021
S31508005210B40200209401002000040048FEF7D2FAE8
S31508005220FDF74AFBFDF7E8F80B20FCF7A3FF09207A
S31508005230FCF7A0FF0420FCF79DFF01215348FDF76A
S3150800524081F94B200002FDF7A1FAFEF757F8FDF7A2
S31508005250CFFFFEF7EDFA0D216320FEF717FB0121BC
S315080052604B48817400214175FFF750FCFEF75AFC44
S315080052707F217E20FEF7F8FE86E04548007C01285F
S3150800528036D1002301221946184600F06BF900238F
S315080052901A461946184600F065F93E4840683E49E0
S315080052A0884204D908213D48FDF7E1FD1DE039494A
S315080052B04868FF21F531FCF72DFBC007C00F002811
S315080052C00ED180210920C006FDF7D1FD082109204D
S315080052D0C006FDF7CCFD01213048FDF7C8FD04E006
S315080052E008210920C006FDF7C4FDFDF7FBF948E0D3
S315080052F02748007C02283AD1FDF74CF9FDF7ACFFA8
S31508005300002301221946184600F02CF900231A46F4
S315080053101946184600F026F91E4840681E49884274
S3150800532004D908211D48FDF7A2FD1DE01949486862
S31508005330FF21F531FCF7EEFAC007C00F00280ED1A1
S3150800534080210920C006FDF792FD08210920C00624
S31508005350FDF78DFD01211148FDF789FD04E00821BF
S315080053600920C006FDF785FDFFF7D0FA09E0FDF72D
S3150800537011F9FFF7A5FEFFF78DF8FDF76DFF00F0B1
S3150800538037FA7E20FEF750FE77E70000002401403A
S31508005390B402002094010020204E000000040048BA
S315080053A0F7B5A0B00C46154680216846FCF7F5FA15
S315080053B0002700267E2168460170FE214170EF21F4
S315080053C081700721C1702099017100214171847192
S315080053D02112C171012101724572291281720126B9
S315080053E005E06846805DC019C7B2701CC6B20B2EB0
S315080053F0F7DBF843401CC1B26846C1727E210173CF
S315080054000D21FEF7FBFB23B0F0BDFFB585B00546C1
S315080054100E460E9F00200190029003900490009083
S3150800542000247E2168460171457186710421C17187
S31508005430079901720899417287723912C17201245B
S3150800544007E001A8015D00980818C0B20090601C2A
S31508005450C4B2082CF5DB0098C043401CC1B26846AC
S3150800546001737E2141730A2101A8FEF7C7FB09B023
S31508005470F0BDF7B584B005460E46002000900190B1
S3150800548002900390002700247E216846017046702A
S3150800549085700121C170694606980871012405E0E6
S315080054A06846005DC019C7B2601CC4B2052CF7DB9C
S315080054B0F843401CC1B2684641717E2181710721BB
S315080054C0FEF79CFB07B0F0BD70B504460D467E207E
S315080054D0FEF7AAFD03E02078641CFEF77FFB28464A
S315080054E0691E8DB20028F6D170BD000030B5A1B096
S315080054F00446802101A8FCF750FA0025002C02D0AA
S31508005500012C20D10FE07E216846017100214171EE
S31508005510442181711321C1711522104902A8FCF793
S3150800552023FA192510E07E2168460171FE21417192
S31508005530442181713321C1713622094902A8FCF739
S3150800554013FA3A2500E000BF00BF802D03DA29468A
S3150800555001A8FFF7B9FF21B030BD000040010020C7
S3150800556055010020FFB583B006460C4617460020B5
S31508005570029000259A480078642803D09948007854
S31508005580642803D101219848817502E000219648D4
S315080055908175002F02D0012F64D164E09348C08E34
S315080055A0A04202D19148C58F00E00525052D01DCF2
S315080055B0052502E0322D00DB0525601BB0420BDD18
S315080055C08948C07E00280DD1884840688749886187
S315080055D001218548C17605E06019B04202DC002148
S315080055E08148C1768048C07E012832D17C4800783F
S315080055F07C490978884203DA0020794908702BE04B
S31508005600601BB0421ADD7948808E642806DB642068
S31508005610734908700121744881751DE07349888EA5
S31508005620C10F091849103C316D4A117010460078AF
S31508005630642811DD6420114608700DE01E2D03DD77
S3150800564064206749087007E02846463064490870B0
S3150800565002E00020624908706148027838460699D7
S31508005660FFF7F2F9B7E0604820300079022808D140
S315080056705E48408DA04202D15C48458F17E00A2556
S3150800568015E0594820300079032808D15748808DFD
S31508005690A04202D15548858F09E00A2507E05348FC
S315080056A0808DA04202D15148858F00E00A25052D3C
S315080056B001DC052502E0322D00DB3225601BB042F5
S315080056C00BDD4948007F002815D1484840684749FE
S315080056D0C8610121444801770DE06019B0420ADC2F
S315080056E04148007F012806D1404840683F49C861C3
S315080056F000213D4801773C48007F01283CD13948C4
S31508005700007837490978884203DA00203549087055
S315080057105AE0601BB0420ADD502032490870012168
S3150800572031488175314840683049C8614CE00521E7
S315080057302846FCF705F92D4949682C4AD269891A81
S3150800574048437D21C9000190FCF7E4F80019B042EE
S315080057500ED950202349087023482038808DB22856
S3150800576032DA0121214828308183FFF75DFA2BE0E0
S3150800577000201C49087027E01C4949681B4AD26961
S31508005780881A7D21C900FCF7C5F8082819D805210B
S315080057902846FCF7D5F815494968144AD269891A82
S315080057A048437D21C9000190FCF7B4F8201AB0429D
S315080057B003D350200B49087006E0002009490870F9
S315080057C002E000200749087006480278384606991C
S315080057D0FFF73AF900BF00BF029807B0F0BD000016
S315080057E0C2000020C3000020B4020020940100205B
S315080057F010B5F748007900285BD00020F5490880E5
S31508005800F3484038408DFF217D31884204DCF0485A
S315080058104038008D88420ADDED482038407D002852
S3150800582005D1ED4948600121E94820384175EA4823
S31508005830006AEA4988420AD9E5482038407D0028A6
S3150800584005D1E54948600121E14820384175E0481D
S315080058502038407D01282CD1DD482038807C01285D
S3150800586027D10023012219461846FFF77BFE00239D
S315080058701A4619461846FFF775FED74840687D212F
S315080058800901884214D90020D34948600821092013
S31508005890C006FDF7ECFA80210920C006FDF7E7FAF5
S315080058A00121CF48FDF7E3FA0021C9482038817461
S315080058B010BDC7482038807C002848D10821092017
S315080058C0C006FDF7D4FA80210920C006FDF7CFFAF5
S315080058D00121C348FDF7CBFA0023012219461846D1
S315080058E0FFF740FE00231A4619461846FFF73AFE08
S315080058F0B9484068FF21F531884204D20421B848E6
S31508005900FDF7B7FA42E27D20C000B349486004219A
S31508005910B348FDF7ACFAAE482038807E002809D196
S315080059200821AF48FDF7A3FA0021A9482038417598
S3150800593041762BE24021AA48FDF790FA0028E1D0EB
S315080059400021A34801710121203881741EE2A04874
S3150800595000790300FEF7C1FB06044AD7FEFDFC49A1
S315080059600023012219461846FFF7FCFD00231A46B4
S3150800597019461846FFF7F6FD95482038007C012899
S3150800598009D1954800699749884203D9002190486A
S31508005990203801748CE7904840687D2109018842C7
S315080059A01FD900208C49486040218D48FDF756FADA
S315080059B0002807D108218A48FDF759FAFF20F53053
S315080059C0FCF73CFF08210920C006FDF750FA8021A4
S315080059D00920C006FDF74BFA01218148FDF747FA71
S315080059E003E008217E48FDF744FACEE17A4840688C
S315080059F0FF21F531884204D204217948FDF739FAA6
S31508005A0003E004217648FDF732FA734948687D2198
S31508005A10C900FBF77FFF23281CD26F4948687D2100
S31508005A20C900FBF777FF192814D969484038018D52
S31508005A306948408D814206DA65484038418D664896
S31508005A40408D814214DB002063494860022160488A
S31508005A5001710DE0604948687D21C900FBF75AFFCE
S31508005A60232805D300205C49486002215848017163
S31508005A7057484038408DFF217D31884204DC544820
S31508005A804038008D88420CDD00230122194618464D
S31508005A90FFF768FD00231A4619461846FFF762FD08
S31508005AA030E04D48418D408F091849484038408DAF
S31508005AB0814210DD642201210846FEF7C5FF012157
S31508005AC0434820388175407E002815D1002140487A
S31508005AD02038417610E04048418D408F09183C48EF
S31508005AE04038408D814207DC01213948203841760B
S31508005AF000220846FEF7A8FF00231A46194618464C
S31508005B00FFF730FD41E134484068FF21F53188420E
S31508005B1004D204213248FDF7ACF903E004213048E9
S31508005B20FDF7A5F92A484038408DFF217D31884286
S31508005B3004DC27484038008D884210DD0023012206
S31508005B4019461846FFF70EFD00231A46194602E0C5
S31508005B50A9E06AE022E01846FFF704FD1DE01E48AA
S31508005B604168008E7D22D200504381420FD21A4AE4
S31508005B70518DFF320132508D01231A46FFF7F2FC90
S31508005B8000231A4619461846FFF7ECFC05E00020E4
S31508005B901149486003210E480171F6E00C48403867
S31508005BA0408DFF217D31884204DC09484038008D4C
S31508005BB0884219DD0023012219461846FFF7D2FC50
S31508005BC000231A4619461846FFF7CCFC2CE00000BD
S31508005BD0D4020020C40000209401002070110100A6
S31508005BE00004004888130000694948687D21C900F7
S31508005BF0FBF790FE6649498E88420FD2644A918D1A
S31508005C00FF320132508D01231A46FFF7ABFC002301
S31508005C101A4619461846FFF7A5FC05E000205C4918
S31508005C20486004215B480171AFE05A484038408D0E
S31508005C30FF217D31884204DC56484038008D884271
S31508005C400CDD0023012219461846FFF78BFC0023BA
S31508005C501A4619461846FFF785FC23E04C4948685A
S31508005C607D21C900FBF756FE4949098F0F3988423D
S31508005C7012D2474AD18EFF320132108D01230022FB
S31508005C80FFF770FC424AD18DFF320132508D012355
S31508005C901A46FFF767FC05E000203D4948600521E4
S31508005CA03C48017171E03A484068FF21F531884265
S31508005CB004D204213848FDF7DCF80FE03448406880
S31508005CC0FF21F531884209D9314840684B21C9007E
S31508005CD0884203D204213048FDF7C9F82C484068A9
S31508005CE02E4988422BD22B484038408DFF21193146
S31508005CF0884204DC27484038008D88420CDD0023A2
S31508005D00012219461846FFF72DFC00231A461946A4
S31508005D101846FFF727FC37E01D4AD18EFF320132BD
S31508005D20108D01230022FFF71DFC194AD18DFF3281
S31508005D300132508D01231A46FFF714FC24E0042192
S31508005D401548FDF796F812484068154988421BD34E
S31508005D5000201449088000210E48017120388174FA
S31508005D600023012219461846FFF7FCFB00231A46B2
S31508005D7019461846FFF7F6FB04210748FDF777F89A
S31508005D8008210548FDF773F800BF00BF00BF8FE57F
S31508005D9094010020D402002000040048A438000022
S31508005DA0983A0000C4000020C85D0008C000002022
S31508005DB0D4000000704100089C5E00089401002091
S31508005DC04C070000804100080000000000000000A9
S31508005DD00000000001020304010203040607080983
S31508005DE000A24A04000000000000000001020304AB
S31508005DF00607080900000000000000000000000077
S31508005E00000000000400000001000000000000007F
S31508005E100000000000000000000000000000000074
S31508005E200000000000000000000000000000000064
S31508005E300000000000000000000000000000000054
S31508005E40000000000000000000011058594C4C30BA
S31508005E503131327878787878787878CB7E00011086
S31508005E6058594C4C30313132787878787878787857
S31508005E7004013205054C4C30313106145941323093
S31508005E803035323848343530343241787878787855
S31108005E907D5D7E000000000000000000A0
S705080018C515
